:020000040800F2
:100000000040042089040008DB030008DD03000829
:10001000DF030008E1030008E3030008E50400082B
:10002000000000000000000000000000E5030008E0
:10003000E703000800000000E9030008EB030008E4
:10004000E5040008E5040008E5040008E5040008EC
:10005000E5040008E5040008E5040008E5040008DC
:10006000E5040008E5040008E5040008E5040008CC
:10007000E5040008E5040008E5040008E5040008BC
:10008000E5040008E5040008E5040008E5040008AC
:10009000E5040008E5040008E5040008E50400089C
:1000A000E5040008E5040008E5040008E50400088C
:1000B000E5040008E5040008E5040008E50400087C
:1000C000E5040008E5040008E5040008E50400086C
:1000D000E5040008E5040008E5040008E50400085C
:1000E000E5040008E5040008E5040008E50400084C
:1000F000E5040008E5040008E5040008E50400083C
:10010000E5040008E5040008E5040008E50400082B
:10011000E5040008E5040008E5040008E50400081B
:10012000E5040008E5040008E5040008E50400080B
:10013000E5040008E5040008E5040008E5040008FB
:10014000E5040008E5040008E5040008E5040008EB
:10015000E5040008E5040008E5040008E5040008DB
:100160000000000000000000E5040008E5040008AD
:10017000E5040008E5040008E5040008E5040008BB
:10018000E5040008E5040008E5040008000000009C
:1001900000000000E504000800000000000000006E
:1001A0000000000000000000E5040008E50400086D
:1001B000E5040008E5040008E5040008E50400087B
:1001C000E5040008E504000800000000000000004D
:1001D000000000000000000000000000E50400082E
:1001E000E5040008E504000800000000000000002D
:1001F000E5040008E5040008E5040008000000002C
:1002000000000000E5040008E5040008E50400081B
:10021000E5040008E5040008E5040008E50400081A
:10022000E50400080000000000000000E5040008EC
:10023000E5040008000000000000000000000000CD
:10024000000000000000000000000000E5040008BD
:04025000E5040008B9
:1002540010B5054C237833B9044B13B10448AFF3FC
:1002640000800123237010BD0C000020000000005A
:100274000013000808B5034B1BB103490348AFF34F
:10028400008008BD000000001000002000130008DA
:1002940010B59CB04C22002109A801F003F81822E3
:1002A400002102A800F0FEFF184B1A6922F0300268
:1002B4001A611A6902F030020192019A5A6911070F
:1002C400FCD50223012408930823CDE90B434023E2
:1002D4000D93002308A8129300F030FD08B172B604
:1002E400FEE71F23CDE90400CDE90230CDE9060085
:1002F400214602A800F0ECFB08B172B6FEE7044AFE
:10030400136823F0300313601CB010BD00080244CE
:1003140000200240002400B589B00021102203A867
:1003240000F0C0FFADF8084000F010FA0123ADF86A
:100334000C306FF07743234A03A8CDE90423224B02
:10034400069300F017FA4FF4884302A8ADF808307A
:1003540000F036FA042000F0E7F900F00BF9FFF79B
:1003640097FFCDE90544194B0C21D3F88C2018488C
:1003740042F00102C3F88C20D3F88C2002F0010271
:100384000192019AD3F88C2042F00202C3F88C2027
:10039400D3F88C3003F002030293029B0223CDE9CD
:1003A4000313072303A9079300F024FA204600F05F
:1003B400C9FA08B172B6FEE700F0D4FA08B172B611
:1003C400FEE7FEE700F0FF0800030100000C024412
:1003D400000002427047FEE7FEE7FEE7FEE7FEE7A5
:1003E40070477047704700F0E9B800001F4910B526
:1003F400D1F888301E4843F47003C1F888301D4B8F
:100404001A6802F0180242F001021A600022DA614E
:100414001A621C682040186017489A62DA621A63EC
:1004240058639A63D8631A6458649A64186820F409
:10043400802018601A654FF000638B600F4B9A6937
:1004440002F04042B2F1404F0FD1DA69D20741BF06
:100454000B4ADA6002F14432DA60DA6942F00202ED
:10046400DA61DA6942F00102DA6110BD00ED00E000
:10047400FBEAE2EA000C024480020101002002408F
:100484003B2A1908DFF83CD00F4880F30A88FFF7AD
:10049400ADFF0E480E490F4A002302E0D458C45061
:1004A4000433C4188C42F9D30B4A0C4C002301E0EA
:1004B40013600432A242FBD300F0FCFEFFF72AFFD4
:1004C400FEE7000000400420003C0420000000205F
:1004D4000C000020301300080C0000202C00002029
:1004E400FEE7000070B5204E054632780AB90120B7
:1004F40070BD4FF0E0231C6914F0040417D04FF4CE
:100504007A73B3FBF2F3194A1468B4FBF3F420468C
:1005140000F0A8F804460028E9D1024629464FF025
:10052400FF3000F06FF8124B20461D60E0E700F04A
:10053400E3F8012807D002280DD00028E7D14FF4B2
:10054400FA533278DDE74FF47A7332784FF4FA4491
:10055400B3FBF2F3D9E74FF47A7332784FF40044E3
:10056400B3FBF2F3D1E700BF040000200000002039
:100574000800002010B5032000F032F800F0FCF968
:100584000B4B0C4A1B6A03F00F03D35CD8400A4B95
:100594001860042000F076F80F20FFF7A3FF04464C
:1005A40018B9FFF717FF204610BD0124FBE700BF71
:1005B400000C02441813000800000020034A044BF6
:1005C40011681B780B441360704700BF280000209B
:1005D40004000020014B1868704700BF2800002069
:1005E40007490302CA6803F4E06322F4E0621204D8
:1005F400120C134343F0BF6343F40033CB607047E2
:1006040000ED00E0154B30B5DC68C4F30224C4F1FE
:100614000703251D042B28BF0423062D4FF0FF35A7
:1006240094BF0024033C05FA03F321EA0303A54025
:1006340022EA0502A340002843EA0203ACBF00F10A
:100644006040074A4FEA0313DBB2ABBF00F56140D9
:1006540000F00F0080F80033135430BD00ED00E0CB
:1006640014ED00E00138B0F1807F3FBF4FF0E0238C
:1006740058610020986137BF1A69012042F00302D3
:100684001A617047042818D8DFE800F00A18261702
:1006940003004FF0E022136943F004031361704731
:1006A4004FF0E022136923F004031361114AD2F8D6
:1006B400E43023F00C03C2F8E43070474FF0E0223A
:1006C400136923F0040313610A4AD2F8E43023F0D7
:1006D4000C0343F00403EEE74FF0E022136923F028
:1006E40004031361034AD2F8E43023F00C0343F00B
:1006F4000803E0E7000C02444FF0E0231B695A07AB
:100704000CD4084BD3F8E40000F00C00042807D004
:10071400A0F1080358425841400070470420704734
:1007240001207047000C0244BFF35F8F064B40F07A
:100734000100C3F894005A6A42F480325A62BFF34B
:100744004F8FBFF36F8F704700ED00E0BFF35F8FF3
:10075400074B5A6A22F480325A62D3F8942022F06A
:100764000102C3F89420BFF34F8FBFF36F8F70471C
:1007740000ED00E0BFF35F8F104A4378C2F8983071
:10078400D2F8A03023F00103C2F8A0304368817B83
:1007940023F01F030B43C17B43EAC103417B43EABC
:1007A4004103C2F89C308368017823F01F030B4394
:1007B400017B43EA4103C2F8A030704700ED00E03A
:1007C40010B5BFF35F8FFF2403784078032B8ABFF3
:1007D40006490749043B0A68DB009C4022EA0402FC
:1007E40000FA03F313430B6010BD00BFC4ED00E037
:1007F400C0ED00E02DE9F74F00234FF00F094F4AF9
:100804004F4C02EA902201920A6832FA03F502D1AF
:1008140003B0BDE8F08F012505FA03F818EA0202D7
:1008240000F08A804D6825F01007022F16D14FEA98
:10083400D30C00EB8C0C03F0070EDCF820604FEABD
:100844008E0E09FA0EFA26EA0A0A0E6906F00F0657
:1008540006FA0EF646EA0A06CCF820600326D0F81B
:1008640000B04FEA430E06FA0EF605F0030A2BEA2F
:10087400060B6FEA060C013F0AFA0EF646EA0B066F
:10088400012F06608E680BD9BAF1030F1AD0C7681E
:1008940006FA0EF60CEA070C46EA0C06C66013E0EC
:1008A40087680CEA070ACF6807FA0EF747EA0A07CF
:1008B4008760476827EA08082F099F4047EA080726
:1008C4004760E4E7012EE2D1EE0035D523F00307BB
:1008D40007F1884803F00306019FF60009FA06FEB3
:1008E40007FA06F6D74308F50838D8F860C015F4B7
:1008F400801F2CEA0E0C46EA0C06C8F860602668D5
:100904000CBF3E4016432660666815F4001F0CBFFA
:100914003E4016436660D4F8846015F4003F0CBF73
:100924003E401643C4F88460D4F88060ED0354BF9D
:100934003E401643C4F88060013365E77F7F2F0093
:10094400002002440146064A106810F0010009BF65
:100954001368012023F004030B4308BF136070479E
:1009640000040340034A0020136843F001031360AA
:10097400704700BF000403404E4B30B5DA6902F003
:100984001802082A00F08F80DA6912F0180F09D1D2
:100994001A68494812F0200F03D01B68C3F3C1033F
:1009A400D84030BDDA6902F01802102A7DD0DA6925
:1009B40002F01802182A7AD1996A9D6A9A6A15F483
:1009C4007C5F9C6BC5F30520EBD0C2F30012C4F32B
:1009D400CC04624307EE900A06EE902A01F003026B
:1009E400012AB8EEE77AFAEEE96AF7EE005A0FD078
:1009F400032A4AD05B6B9FED316AC3F3080307EE09
:100A0400903AF8EEE77A77EEA67A77EEA57A37E0B1
:100A14001A68920627D51968274AC1F3C101CA404A
:100A240007EE902AB8EEE76A5B6BC6EE077AC3F36B
:100A3400080307EE103AB8EEC77A37EE267A37EE97
:100A4400257A67EE877A1B4B5B6BC3F3462301332E
:100A540007EE103AF8EEC76A87EEA67AFCEEC77A7C
:100A640017EE900A9DE75B6B9FED156AC3F30803CD
:100A740007EE903AF8EEE77A77EEA67A77EEA57A63
:100A8400C6EE076A67EEA67ADDE75B6B9FED0D6A3B
:100A9400C3F3080307EE903AF8EEE77A77EEA67A06
:100AA40077EEA57AECE708487BE7084879E702483F
:100AB40077E700BF000C02440090D0030024744A7E
:100AC4000024744C20BCBE4B00093D0040787D01DD
:100AD4002DE9F0410D46044610B90120BDE8F0812E
:100AE400864A136803F00F038B426FD32368DE0634
:100AF40078D418070DD5824920690A6A120902F0D0
:100B04007002904281BF0A6A22F4E06242EA001253
:100B14000A6259070BD57A49E0680A6A02F0700242
:100B2400904281BF0A6A22F0700202430A629A0765
:100B34000BD57349A0680A6A02F00F02904281BF84
:100B44000A6A22F00F0202430A62DF0759D42268BC
:100B5400960700F1AC8069490B6803F00F03AB42C0
:100B640000F2B280500700F1BB8011070DD5644933
:100B740020690B6A1B0903F0700398423FBF0B6A9C
:100B840023F4E06343EA00130B62D3060DD55C4AF9
:100B94006169136A1B0A03F0700399423FBF136A29
:100BA40023F4E04343EA01231362FFF7E5FEBDE8C3
:100BB400F041534B534A1B6A03F00F03D35CD840F4
:100BC400514B1860514B1868FFF78CBC136823F025
:100BD4000F030B431360136803F00F038B427FF47E
:100BE4007CAF83E7464960690A6A120A02F0700220
:100BF400904281BF0A6A22F4E04242EA00220A6279
:100C040077E761683E4B03291A681DD112F0007F13
:100C14003FF463AFDA6941F2883822F003020A43F1
:100C2400DA61FFF7D7FC63680646032B344F18D10B
:100C3400FB6903F01803182B89D0FFF7CBFC801B4A
:100C44004045F5D9032049E7022902D112F4003FB7
:100C5400DEE7012902D112F4007FD9E712F0020F76
:100C6400D6E7022B0BD1FB6903F01803102B3FF4DA
:100C74006EAFFFF7AFFC801B4045F4D9E2E7012BD0
:100C840010D1FB6903F01803082B3FF460AFFFF7A2
:100C9400A1FC801B4045F4D9D4E7FFF79BFC801BE3
:100CA4004045CFD8FB6913F0180FF6D14FE714492C
:100CB400A0680B6A03F00F0398423FBF0B6A23F04E
:100CC4000F0303430B6246E70B6823F00F032B4328
:100CD4000B600B6803F00F03AB427FF4FEAE41E7F9
:100CE4000749E0680B6A03F0700398423FBF0B6A40
:100CF40023F0700303430B6237E700BF0020024078
:100D0400000C024418130008000000200800002012
:100D140008B5FFF731FE064B064A1B6A03F00F03C2
:100D2400D35C03F01F03D840034B186008BD00BF19
:100D3400000C024418130008000000202DE9F041C3
:100D4400044600286AD0994BDE699F6A036806F05E
:100D54001806DA0607F0030710D5082EC36903D076
:100D6400182E24D1022F22D1002B57D08F4A216A6A
:100D7400936923F47C1343EA014393612368D907FD
:100D840043D423689A0700F19E8023681D0700F16D
:100D9400F6802368580700F1218123689B0600F13F
:100DA4009A81A16A002940F0BB8100201AE07F4D9E
:100DB400D3B12B6843F480732B60FFF70BFC8046A0
:100DC4002B689B0507D5AB69226A23F47C1343EA9D
:100DD4000243AB61D2E7FFF7FDFBA0EB080002285A
:100DE400EED90320BDE8F0812B6823F480732B60D7
:100DF400FFF7F0FB80462B689805BFD5FFF7EAFBA9
:100E0400A0EB08000228F6D9EBE7102E636803D0A4
:100E1400182E05D1032F03D1002BB2D10120E1E715
:100E2400B3F5803F614D12D12B6843F480332B60BE
:100E3400FFF7D0FB0546DFF87481D8F800309B0338
:100E44009FD4FFF7C7FB401B6428F6D9C9E7C3B991
:100E54002B6823F480332B602B6823F480132B60DE
:100E64002B6823F480232B60FFF7B4FB80462B68A8
:100E7400980386D5FFF7AEFBA0EB08006428F6D9EB
:100E8400AFE7B3F5A02F08D12B6843F480232B6080
:100E94002B6823F480132B60C6E7B3F5A81F2B68D7
:100EA40006D143F480232B602B6843F48013F2E7CC
:100EB40023F480332B602B6823F480232B602B686E
:100EC40023F48013B3E7E3681EB1182E2ED1012F4B
:100ED4002CD1002BA2D076B1FFF77CFB0746334D13
:100EE4002B6899071CD52B69626923F4FE0343EA36
:100EF40002432B6149E72D4A2169136803F0180363
:100F04008B42E9D0136823F018030B431360FFF7F7
:100F1400FFFE274B1868FFF7E5FA0028DCD07DE7D1
:100F2400FFF758FBC01B0228DAD95AE71F4DABB1B3
:100F34002B68226923F0180313432B602B6843F0BA
:100F440001032B60FFF746FB07462B689A07CAD4B8
:100F5400FFF740FBC01B0228F7D942E72B6823F0B8
:100F640001032B60FFF736FB07462B689B077FF5D1
:100F74000CAFFFF72FFBC01B0228F6D931E7A3699A
:100F84000A4DBBB1D5F8F03043F08063C5F8F030BA
:100F9400FFF720FB0746D5F8F03019013FF5F9AE0D
:100FA400FFF718FBC01B0228F5D91AE7000C02440E
:100FB40008000020D5F8F03023F08063C5F8F03045
:100FC400FFF708FB0746D5F8F0301A017FF5E1AECC
:100FD400FFF700FBC01B0228F5D902E7AF4D6B6A8F
:100FE400DF071AD5A368AE4D012B26D1D5F8F03012
:100FF40043F00103C5F8F030FFF7ECFA41F288380A
:101004000546A74FD7F8F03099073FF5C6AEFFF76E
:10101400E1FA401B4045F5D9E3E66B6A43F001036E
:101024006B62FFF7D7FA07466B6AD807DAD4FFF783
:10103400D1FAC01B0228F7D9D3E60BBBD5F8F030A0
:1010440041F2883823F00103C5F8F030D5F8F030C8
:1010540023F08003C5F8F030D5F8F03023F0040312
:10106400C5F8F030FFF7B6FA0746D5F8F0309A071E
:101074007FF593AEFFF7AEFAC01B4045F5D9B0E655
:10108400052B0CD1D5F8F03043F00403C5F8F0304B
:10109400D5F8F03023F08003C5F8F030A6E7852BAF
:1010A400D5F8F03008D143F00403C5F8F030D5F892
:1010B400F03043F08003EFE723F00103C5F8F0308C
:1010C400D5F8F03023F00403C5F8F030D5F8F0304B
:1010D40023F080038EE7636A714D83B12B6843F478
:1010E40080532B60FFF776FA07462B689B043FF585
:1010F40058AEFFF76FFAC01B0228F6D971E62B68C9
:1011040023F480532B60FFF765FA07462B68980495
:101114007FF547AEFFF75EFAC01B0228F6D960E6FA
:10112400182E5F4D72D02B68022923F080732B6038
:1011340059D1FFF74FFA06462B6899014DD4AB6A93
:10114400E26A23F47C5323F003031343226B43EA40
:101154000223AB62A36BE26B013B013A5B02120414
:1011640002F4FE029BB21343626B013AC2F308021B
:101174001343226C013A120602F0FE4213436B63DE
:10118400AB6A23F01003AB62E36CDB00AB63AB6AC6
:1011940043F01003AB62AB6A626C23F00C0313439D
:1011A400AB62AB6AA26C23F020031343AB62AB6A5D
:1011B40043F48033AB622B6843F080732B60FFF7FA
:1011C40009FA0446364D2B689A013FF5EEADFFF758
:1011D40001FA001B0228F6D903E6FFF7FBF9801B8E
:1011E4000228A9D9FDE5FFF7F5F904462B689B0110
:1011F40006D4AB6A23F4E02323F00303AB62D4E503
:10120400FFF7E8F9001B0228F0D9EAE50129AA6AE8
:101214006B6B3FF403AEE06A02F0030181427FF49A
:10122400FDAD216BC2F305228A427FF4F7AD626BF8
:10123400C3F30801013A91427FF4F0ADA26BC3F30A
:101244004621013A91427FF4E9ADE26BC3F30641D2
:10125400013A91427FF4E2AD226CC3F30663013A92
:1012640093427FF4DBADAB6BE26CC3F3CC039342EC
:101274003FF49BAD0A4DAB6A23F01003AB62FFF75A
:10128400A9F90646FFF7A6F9B042FBD0E36CDB00F0
:10129400AB63AB6A43F01003B0E700BF000802443D
:1012A400000C024402440346934200D1704703F801
:1012B400011BF9E770B50D4B00260D4D5B1B9C100F
:1012C400A64209D10B4D00F019F80B4B00265B1B0D
:1012D4009C10A64205D170BD55F8043B01369847D1
:1012E400EEE755F8043B01369847F2E72813000867
:1012F40028130008281300082C130008F8B500BFB1
:10130400F8BC08BC9E467047F8B500BFF8BC08BCE2
:041314009E4670473A
:10131800000000000000000001020304060708099D
:04132800790200083E
:04132C00550200085E
:0C1330000090D00301000000100000003D
:040000050800048962
:00000001FF
